:100000000C9435000C945D000C945D000C945D0024
:100010000C945D000C945D000C945D000C945D00EC
:100020000C945D000C945D000C945D000C945D00DC
:100030000C945D000C945D000C945D000C945D00CC
:100040000C9486000C945D000C9408010C945D00E7
:100050000C945D000C945D000C945D000C945D00AC
:100060000C945D000C945D008D0211241FBECFEF37
:10007000D8E0DEBFCDBF11E0A0E0B1E0EAEBF8E0F0
:1000800002C005900D92AA30B107D9F711E0AAE09D
:10009000B1E001C01D92AA3AB107E1F710E0CAE64B
:1000A000D0E004C02297FE010E945704C836D10751
:1000B000C9F70E947F000C945B040C9400000FC0F1
:1000C00087E991E00E945202AC01662757FD6095D6
:1000D000762F87E991E020E030E00E94BD0387E9B8
:1000E00091E00E943E02882359F7089587E991E044
:1000F00040E855E260E070E00E94450108950E94EA
:10010000CE000E9476000E945F00FDCF1F920F92EA
:100110000FB60F9211242F933F938F939F93AF931A
:10012000BF9380910E0190910F01A0911001B091A9
:100130001101309112010196A11DB11D232F2D5FD8
:100140002D3720F02D570196A11DB11D20931201CE
:1001500080930E0190930F01A0931001B0931101B1
:1001600080910A0190910B01A0910C01B0910D01B9
:100170000196A11DB11D80930A0190930B01A093DC
:100180000C01B0930D01BF91AF919F918F913F9161
:100190002F910F900FBE0F901F901895789484B5F3
:1001A000826084BD84B5816084BD85B5826085BD73
:1001B00085B5816085BDEEE6F0E080818160808359
:1001C000E1E8F0E0808182608083808181608083CB
:1001D000E0E8F0E0808181608083E1EBF0E0808105
:1001E00084608083E0EBF0E0808181608083EAE7D7
:1001F000F0E0808184608083808182608083808160
:10020000816080838081806880831092C10008951E
:100210001F920F920FB60F9211242F933F934F937B
:100220005F936F937F938F939F93AF93BF93EF935E
:10023000FF934091C600E0919301F0919401CF01AA
:10024000019660E870E00E94F1039C0180919501A5
:10025000909196012817390739F0ED5EFE4F4083E3
:100260003093940120939301FF91EF91BF91AF914F
:100270009F918F917F916F915F914F913F912F91BE
:100280000F900FBE0F901F9018955F926F927F9204
:100290008F929F92AF92BF92CF92DF92EF92FF9296
:1002A0000F931F93CF93DF93EC013A014B0141343D
:1002B00082E458078FE0680780E078070CF07FC081
:1002C00060E874E88EE190E0A40193010E942604A6
:1002D0002150304040405040CA01B90122E030E096
:1002E00040E050E00E94260459016A01A6019501F0
:1002F000209530954095509594E0220F331F441F70
:10030000551F9A95D1F760E074E284EF90E00E9467
:100310002604CA01B9012FEF30E040E050E00E940E
:10032000D203A40193010E942604C90181509F4F6A
:10033000181619061CF4522E5A9403C055245394CF
:10034000521A60E079E08DE390E0A40193010E94ED
:1003500026042150304040405040CA01B90122E0FB
:1003600030E040E050E00E94260420953095409512
:10037000509583E0220F331F441F551F8A95D1F7F4
:1003800060E074E284EF90E00E942604CA01B901A3
:100390002FEF30E040E050E00E94D203A40193012F
:1003A0000E942604C90181509F4F181619061CF49B
:1003B000822F815002C081E0821B851500F5E885FF
:1003C000F98581E090E00A8802C0880F991F0A949D
:1003D000E2F7808360E079E08DE390E0A40193018F
:1003E0000E9426042150304040405040CA01B901CB
:1003F00022E030E040E050E00E94260404C0E8859E
:10040000F98510829501EC81FD813083EE81FF81B9
:100410002083EA85FB85208141E050E0CA010E84FB
:1004200002C0880F991F0A94E2F7282B2083EA85DF
:10043000FB852081CA010F8402C0880F991F0A948E
:10044000E2F7282B2083EA85FB858081088802C09B
:10045000440F551F0A94E2F7842B8083DF91CF91DC
:100460001F910F91FF90EF90DF90CF90BF90AF90D2
:100470009F908F907F906F905F900895DC0112960F
:10048000ED91FC911397E058FF4F81919191805825
:100490009F4F20813181821B930B60E870E00E94A6
:1004A000F1030895CF93DF93DC011296ED91FC9157
:1004B0001397EF01CE57DF4F48815981E058FF4F26
:1004C00080819181E058F0408417950719F42FEF4F
:1004D0003FEF0CC0E40FF51F2081CA01019660E8D0
:1004E00070E00E94F1039983888330E0C901DF91B5
:1004F000CF910895FC01A085B18521898C9190E070
:10050000022E02C0959587950A94E2F780FFF6CFF8
:100510000484F585E02D6083089584E091E0909354
:1005200098018093970183E191E090939A018093E1
:10053000990185EC90E090939C0180939B0184EC61
:1005400090E090939E0180939D0180EC90E09093C9
:10055000A00180939F0181EC90E09093A201809391
:10056000A10186EC90E09093A4018093A30184E024
:100570008093A50183E08093A60187E08093A70183
:1005800085E08093A80181E08093A90108950F93ED
:100590001F93CF93DF938C01EB0109C02196D80103
:1005A000ED91FC910190F081E02DC80109956881E1
:1005B0006623A1F7DF91CF911F910F910895EF92DC
:1005C000FF920F931F93CF93DF938C017B01EA017E
:1005D0000CC0D7016D917D01D801ED91FC91019086
:1005E000F081E02DC80109952197209791F7DF91BF
:1005F000CF911F910F91FF90EF9008952F923F920E
:100600004F925F926F927F928F929F92AF92BF9222
:10061000CF92DF92EF92FF920F931F93DF93CF93CE
:10062000CDB7DEB7A0970FB6F894DEBF0FBECDBF33
:100630001C016A017B01411551056105710549F4F1
:10064000DC01ED91FC910190F081E02D60E30995D2
:1006500054C0882499245401422E552466247724BA
:1006600001E010E00C0F1D1F080D191DC701B60198
:10067000A30192010E940404F80160830894811C84
:10068000911CA11CB11CC701B601A30192010E94DB
:100690000404C901DA016C017D01C114D104E10433
:1006A000F104F1F681E0E82EF12CEC0EFD1EE80CD1
:1006B000F91C3E010894611C711CD501C40101970D
:1006C000A109B1096C01C818D90814C0F601EE0DD2
:1006D000FF1D60816A3010F4605D01C0695CD1016A
:1006E000ED91FC910190F081E02DC10109950894F4
:1006F000E108F1086E147F0449F7A0960FB6F8944C
:10070000DEBF0FBECDBFCF91DF911F910F91FF9044
:10071000EF90DF90CF90BF90AF909F908F907F90A1
:100720006F905F904F903F902F900895EF92FF92BF
:100730000F931F93CF93DF93EC017A018B0177FF27
:100740000FC0E881F9810190F081E02D6DE20995FB
:1007500010950095F094E094E11CF11C011D111D11
:10076000CE01B801A7012AE00E94FE02DF91CF91DD
:100770001F910F91FF90EF900895DC012115310535
:1007800041F4ED91FC910190F081E02D642F0995E9
:1007900008952A30310519F40E94960308950E94A5
:1007A000FE020895629FD001739FF001829FE00DC9
:1007B000F11D649FE00DF11D929FF00D839FF00DE0
:1007C000749FF00D659FF00D9927729FB00DE11D8C
:1007D000F91F639FB00DE11DF91FBD01CF01112469
:1007E000089597FB092E07260AD077FD04D049D03B
:1007F00006D000201AF4709561957F4F0895F6F7A2
:10080000909581959F4F0895A1E21A2EAA1BBB1BBC
:10081000FD010DC0AA1FBB1FEE1FFF1FA217B307CC
:10082000E407F50720F0A21BB30BE40BF50B661FE2
:10083000771F881F991F1A9469F7609570958095A6
:1008400090959B01AC01BD01CF01089597FB092E46
:1008500005260ED057FD04D0D7DF0AD0001C38F48F
:1008600050954095309521953F4F4F4F5F4F0895DC
:10087000F6F790958095709561957F4F8F4F9F4FBC
:100880000895AA1BBB1B51E107C0AA1FBB1FA617D7
:10089000B70710F0A61BB70B881F991F5A95A9F729
:1008A00080959095BC01CD010895EE0FFF1F059036
:0A08B000F491E02D0994F894FFCFB5
:0A08BA00000000007A02C702DF020E
:00000001FF
